:020000040000FA
:020000000528D1
:08000800A32C031383129F01D6
:10001000831606309F003F30850086018701083037
:1000200088008901803081000C108312013090001B
:10003000860140308700071388018901C401051C2F
:10004000441410240C30E6230230AD00FD30AE0025
:100050004824C030E62348240B178B176F24053043
:10006000A1008030860087160000871295240717AC
:100070000000071389149524891009159524091186
:10008000A10B31289D240130E6230330AD001F3041
:10009000AE004824C030E62348249D240130E623E6
:1000A0009D249B240130E6230330AD004130AE0097
:1000B0004824C030E62348246F249B24A2010D303D
:1000C000E6232208B620A6008038E623051C6D280A
:1000D000851C9623051DA42361289B240130E6235B
:1000E0003C30E8230330AD004130AE002608A700C5
:1000F000271F8028BF30A7050330AD005230AE0067
:10010000A70AAE0A0319AD0AA70B812853248A1146
:100110000A12E82353248A110A12AE0A0319AD0AFF
:100120004B3C031D86283E30E8230D30E623883003
:10013000E6230330AD006330AE0048246F249B24D7
:1001400005080F390F3AA500A5195128251CA0282C
:10015000BF01C0016F24A51CAF283F14B328251D83
:10016000B3284014A50144184529C528C03EAE0057
:1001700000300318013EAD0053248A110A12080012
:1001800007340D34403446344B342208A300053084
:10019000A4002403A20023082202031C3029220801
:1001A000B22302224508B6004608B7000130B50068
:1001B0004922FF30B9006D220130C3008F22B808F8
:1001C000031929290030220203192C290830B60608
:1001D0004922B9016D220830B60449220130C3001A
:1001E0008F22B8080319292904302202031D062989
:1001F000B5014922B9016D220130B5004922013013
:10020000C3008F22B808031929292C2903302202A0
:10021000031D19298030B6064922B9016D228030AC
:10022000B60449220130C3008F22B80803192929D6
:100230002C2902302202031D2C292030B606492227
:10024000FF30B9006D220130C3008F22B808031DB2
:100250002C29A40BC9283029230822023E10031D93
:100260003E142308A2003E1C45290717000007136F
:10027000C030E6230330AD006B30AE0048240915D2
:100280007C240518412989016E280C30E62388302A
:10029000E6230330AD007C30AE004824C030E623B6
:1002A0004824B2230222C301881D4314BC01BD01AE
:1002B000BE0140185F29050E0339033AA50021222B
:1002C0002508031D7629B601B701B5013622B9010B
:1002D00066228F22B1224118E629851DE629B90F31
:1002E0006829CE22C20803196629E62901302502B1
:1002F000031D9529B901B601B701B5013622662261
:10030000CE22C20803197E29B601B701B5013622F3
:100310008F22B1224118E629851DE629CE22C20886
:1003200003198729B90F7B29E62902302502031D0D
:10033000C829BA01B601B701B5013A08B900362299
:100340006622CE22C208031DA729B90A9F29B60139
:10035000B701B5013A08B90036228F22B1224118FF
:10036000E629851DE629CE22C208031DB929B90A4E
:10037000AC29BA0F9A29E62901340234043408342E
:1003800010342034403480340034FF345534AA34DF
:10039000B601B701B50136220130AD00BC30AE0068
:1003A00053248A110A12AE0A0319AD0AB900662253
:1003B0008F22B1224118E629851DE629AA3039028B
:1003C000031DD029CE22C2080319CB29BE08031968
:1003D000EC2909157C24EE298914742407170000E0
:1003E00007134018F7290518F32989016E28851D80
:1003F000F5290519F7298901A50A04302502031DED
:1004000045296E280630BB0403302202031C0A2A49
:100410000830BB043B0886008716000087122208BC
:10042000031D182A08308600071500000711202A2E
:10043000013C031D202A203086000715000007110B
:100440000800023022020330031C2C2A043022024E
:100450000430031C2C2A05308038E6232C30E82396
:1004600031302507E8233E30E8230800C308031D88
:10047000492AC230E6233608E8223708E822043049
:100480002202031D492AC130E6230F303505F2222E
:10049000E8232208031D4E2A0830532A013C00306D
:1004A000031D532A2030360486000715000007116B
:1004B0003708860087150000871104302202031DCB
:1004C000652A07103508031D07140800C308031D1B
:1004D0006D2AC930E6233908E822390886008714D6
:1004E00000008710A208031D822A360807398600FB
:1004F00007150000071136080838860007150000A8
:1005000007118E2A3B113B088600871600008712D0
:100510003B153B0886008716000087120800071667
:10052000BB103B0886008716000087120313831652
:10053000FF308600831287170608B80087138316DA
:1005400086018312BB143B088600871600008712C1
:100550000712C308031DB02ACE30E6233808E8226C
:100560000800C101380839020319CD2ABD0A031950
:10057000BC0A3E148C30E6233C08E8223D08E82201
:10058000BF080319CD2A091557248519C92A411412
:10059000CD2A0519C52A09119B240800C201460865
:1005A0003702031DD72A450836020319DB2AB70A8A
:1005B0000319B60AE72A04302202031DE62AB50809
:1005C000031DE62AB50AB601B701E72A421408005E
:1005D000C900490E0F39F222E8230F304905F222F3
:1005E000E8230800CA000A3C0319FA2A031CFA2A65
:1005F0003030FB2A37304A070800533474346134F2
:10060000743469346334523461346D34433468343F
:10061000653463346B3465347234003420342034F0
:10062000203428342034383420346234693474342B
:100630002034293420342034203420340034203431
:100640002034203420347634653472342E343134FE
:100650002E343034373420342034203420340034E5
:10066000203420346234793420346D342E3479349B
:1006700061346D3461346D346F3474346F342034CC
:10068000003454347934703465343F345F3420346A
:10069000203432344B342034203420342034383465
:1006A0004B3400342034333432344B34203420344F
:1006B0002034363434344B34203420343134323422
:1006C00038344B34003453347434613472347434F9
:1006D0003F345F340034543479347034653420341A
:1006E0004D34693473346D34613474346334683434
:1006F00020342134213400342034453472343A34E7
:100700003034303430343034003441343A342034EE
:10071000203420342034203457343A3420342034E8
:10072000203452343A342034203400341E3096249D
:100730008518A32B692496309624A203220A031D50
:10074000A32B0430A20008001E3096240519B12BFB
:10075000692496309624A20A05302202031DB12B8B
:10076000A20108000330AD00D730AE002208C70058
:10077000C7080319C42B0330C800AE0A0319AD0A19
:10078000C80BBD2BC703B82B53248A110A12BB0018
:10079000AE0A0319AD0A53248A110A12C500AE0A23
:1007A0000319AD0A53248A110A12C6000800203426
:1007B0000734FF3440341F34FF3440347F34FF3477
:1007C0008034FF34FF348034FF34FF340811EA2BC7
:1007D000081500008810F023200EF023FA230800EB
:1007E000A0000F308805F0302005880408140000B0
:1007F000081008008316F0308804831208110000E6
:100800008814081408080810A00008140808081024
:10081000A01B012C88108316F03088068312080074
:10082000881000000811000008100F3096243030A6
:10083000F023053096243030F02389243030F02323
:1008400089242030F02389242830E6230830E62349
:100850000130E6230630E62308008316F0308804D2
:100860008312081500008814081408080810F039CD
:10087000A000A00E081408080810F039A004A00E6B
:1008800088108316F0308806831289242008080017
:1008900053248A110A12AE0A0319AD0A003E031945
:1008A0000800E823482C2D088A002E088200DA3040
:1008B000AF00AD30B000FA30812CDA30AF00AD308F
:1008C000B0004630812CE730AF001730B000463022
:1008D000812CED30AF005730B0004630812C6324BE
:1008E0001E309624692408000430B40069241E30A8
:1008F0009624B40B762C08005D24463096245724A9
:10090000080083160C148312962483160C1083128D
:1009100008006330B1008C2CB10B8B2C08000A301E
:10092000B2008924B20B912C08006430B3008F24EC
:10093000B30B972C080005309E2C0F30B400952483
:10094000B40B9F2C0800F0000308F100831203137E
:100950000C1CB12C2F088F0030088E000130890646
:0C0960000C1071088300F00E700E0900EE
:02400E00323F3F
:1042000043006F0070007900720069006700680069
:1042100074002000280043002900200032003000F4
:10422000310030002D003200300031003800200015
:104230006200790020004D002E00590061006D00E1
:0A42400061006D006F0074006F0054
:00000001FF
